:1000000065C0D4C17EC07DC07CC07BC07AC079C0D1
:1000100078C077C076C075C074C073C072C071C03C
:1000200070C06FC06EC00902220001010080320959
:100030000400000103000000092101010001220069
:10004000000705810308000A04030904180372006D
:100050006100700068006E00650074002E006E0084
:10006000650074001603470043002F004E00360061
:1000700034005F005500530042000A033100300095
:1000800030003000120101010000000881179A0AB7
:1000900002010102030105010905A1010901A100F5
:1000A00005010930093109330934093509361500CC
:1000B00026FF00750895068102C00509190129105F
:1000C00015002501750195108102C00011241FBE85
:1000D000CFE5D4E0DEBFCDBF10E0A0E6B0E0E4E0C5
:1000E000F1E102C005900D92A239B107D9F710E0F5
:1000F000A2E9B0E001C01D92AE3FB107E1F73CD3E9
:10010000FFC77ECF82E990E08093F2000B96809348
:10011000E60085B7836085BF8BB780648BBF089589
:100120000F931F938091F700882309F4A5C0482FEF
:10013000435047FD9FC022E930E09091E6009F5F69
:100140008091F4008D3209F08DC0483009F08AC0EA
:10015000E92FF32F8081807609F07FC01092E100B3
:100160008181882339F41092E20081EE90E030E83A
:1001700022E068C0853021F482818093F8005EC05F
:10018000863009F045C08381813039F42091F9002F
:100190008091E4009091E50039C0823029F486E234
:1001A00090E030EC22E24EC08330E9F48281882373
:1001B00029F488E490E030EC24E044C0813029F454
:1001C0008CE490E030EC28E13DC0823029F484E6F4
:1001D00090E030EC26E136C0833071F48AE790E09D
:1001E00030EC2AE02FC0813229F488E390E030EC33
:1001F00029E028C0823221F081EE90E030EC21C06D
:100200002091E3008091FC009091FD0030EC1AC039
:10021000883019F48BEF90E00AC0893021F4828194
:100220008093FB000BC08A3029F481EE90E030E827
:1002300021E008C08B3011F41092AA0081EE90E00A
:1002400030E820E09093F6008093F50087818823C2
:1002500061F48681821750F008C0892F932F5CD2F9
:1002600030E804C030E880E001C0822F3093A8005D
:10027000809360001092F700909160009F3F09F416
:100280004FC08091610087FF4BC0192F993008F053
:1002900018E0911B909360008091A80080FD02C03F
:1002A0000BE401C003EC8F5F8093A8002091F50060
:1002B0003091F60086FD05C0D901912FE9EDF0E0FF
:1002C00018C04091E300A9EDB0E0F901812F0BC007
:1002D000949150E0EF33F50711F44C9301C09C93D7
:1002E000319681501196882399F705C08D9181939D
:1002F00091509923D9F7C901810F911D9093F60070
:100300008093F50089ED90E0612F02D2183019F04A
:100310008FEF809360000093D8001C5F1093610002
:1003200080B3857019F01092A90011C08091A900C6
:10033000882369F494E680B3857049F49150D9F725
:1003400081E08093A9001092F8001092F3001F91B1
:100350000F9108951F93DC01162F693008F018E003
:100360009091AA0090FD02C02BE401C023EC809183
:10037000620087FF04C09F5F9093AA0003C08FEFC5
:10038000809362002093E700912FE8EEF0E003C035
:100390008D91819391509923D9F788EE90E0612F48
:1003A000B7D11C5F109362001F9108950F930FB790
:1003B0000F93809BFECF809B06C0809B04C0809BD8
:1003C00002C0000000C01F933F932F9331E014E060
:1003D00000B3102710FD32E0102F3A95C9F700FD49
:1003E000E7C000B3102717952FE72795DF9310B3C9
:1003F000012707952795CF93C091F20000B31027EE
:10040000179527953BE0D0E04F9310B30127079550
:1004100027954FEF000055C0809BFECF809B06C004
:10042000809B04C0809B02C0000000C0DF9100C020
:10043000CDCF10B3157079F1407C2C6F13C000B391
:10044000057049F141782C6F15C0057021F1102F0E
:100450002C6F00B319C000B30570E9F04E7F2C6F0C
:1004600018C038F300B30570B1F010271795279521
:10047000243028F310B30127079527954227499385
:100480004FEF00B3243008F3102717952795243039
:1004900010F310B31570E1F101270795279524306B
:1004A000F0F000B30570A1F11027179527952430BF
:1004B000E0F010B30127079527953A9541F12430D4
:1004C000D0F000B3057021F110271795279524303F
:1004D000C0F010B30127079527952430C2CF10B381
:1004E0001570B1F04C7F2C6FDCCF00B3057081F03C
:1004F000487F2C6FDECF10B3157051F0407F2C6F0A
:10050000E0CF00B3057021F0407E2C6FE2CF3DC0FC
:100510003C2FC091F2003C1B00E433300ABFA8F12D
:1005200008811981412F1F772091F3000D3289F145
:10053000013E79F10936C1F00777033431F51091A6
:10054000FA00112311F10091F7000030D1F5343099
:10055000DAF13093F7001093F4000091E600C093B5
:10056000E6000093F20030C0121779F447FD3AC05C
:10057000309161003F3F29F10FEF00936100C8ED1A
:10058000D0E025C000270093FA004F91CF91DF9172
:100590000FC01217B9F70093FA000FEF0093600035
:1005A000009361004F91CF910AB706FD35CFDF91DF
:1005B00000E40ABF2F913F911F910F910FBF0F9140
:1005C0001895C4E6D0E002C0C3E6D0E032E05F9305
:1005D00002B30A7F016002BB55E011B3156011BB85
:1005E00020E819C0309162003F3F59F30FEF0093AC
:1005F0006200C7EED0E0EBCF052710E002BB10C0D1
:10060000052710E0089402BB13C0052710E015C0B1
:10061000052710E019C020FF052702BB2795179575
:100620001C3F50F720FF0527279502BB17951C3F5D
:1006300038F720FF05272795179502BB1C3F28F7A1
:1006400020FF0527279517951C3F02BB08F700C020
:10065000499120FF052702BB279517951C3F80F580
:1006600020FF0527279502BB17951C3F68F520FF43
:1006700005272795179502BB1C3F58F520FF052736
:10068000279517951C3F02BB38F5242F3A9519F68C
:100690000A7F5F9102BB32E03A95F1F71091F800C2
:1006A000C656D04011F01093F300016011B31A7FC9
:1006B00002BB0A7F4F91CF9111BB02BBDF9178CF74
:1006C000052710E002BBCACF052710E0089402BB43
:1006D000CDCF052710E0CFCF052710E0D3CFA82F2F
:1006E000B92F8FEF9FEF41E050EA615070F02D91EC
:1006F00038E0722F782796958795269570FF02C06F
:10070000842795273A95A9F7F0CF8095909508957D
:10071000E6DF8D939D930895FC012DEA30E0309340
:10072000F6002093F50080818076803219F5818172
:10073000813079F4E091AB00F091AC000088F18950
:10074000E02DC9010995E091AB00F091AC008081EA
:100750000895823041F485EB90E09093F600809309
:10076000F50081E008958A3029F483818093B500F3
:1007700080E0089580E00895CF92DF92EF92FF929B
:100780000F931F9314BA8FEF85BB88EF82BB85E070
:1007900081BBE8EEF0E83197F1F711BA83BF8FE043
:1007A00085BD84EC83BD0CE211E0F4D2FC01909392
:1007B000AC008093AB000284F385E02D0995E091B5
:1007C000AB00F091AC000288F389E02D09958823F5
:1007D00019F58CE291E0F8013197F1F70197D9F71B
:1007E00071D4FC019093AC008093AB000284F3853C
:1007F000E02D0995E091AB00F091AC000288F389FF
:10080000E02D0995882341F48CE291E0F8013197BD
:10081000F1F70197D9F7C9CF86E990E09093FD00F1
:100820008093FC005DD48093E30084E890E0909393
:10083000E5008093E400BCD28093F90014BA8FEFF6
:1008400085BB88EF82BB85E081BBE8EEF0E831979D
:10085000F1F711BA83BF1FE015BD84EC83BDE091B1
:10086000AB00F091AC000284F385E02D099588E19E
:1008700090E00FB6F894A89581BD0FBE11BD42DC83
:100880007894FF2401E010E0CC24C39490E8D92EA2
:1008900004C0FF24F39400E01E2DA89541DC002342
:1008A00041F0E091AB00F091AC000484F585E02DBF
:1008B000099508B600FE0EC0C8BEE090B500EE2057
:1008C00049F0153018F4FF24F39405C08BEFE82E9F
:1008D000E10E01C0E12E08B607FE16C0D8BEFF200B
:1008E000A9F4E091AB00F091AC000484F585E02D13
:1008F0000995E091AB00F091AC000684F785E02DFE
:100900000995882319F4C7CFFF2029F2809162004E
:100910008F3F09F0BECFE091AB00F091AC000088B2
:10092000F189E02D8DEA90E00995E091AB00F0911E
:10093000AC008DEA90E060810DDDFF24ACCF009724
:1009400041F0DC01E6EBF0E088E001900D9281508F
:10095000E1F7AEEBB0E0E6EBF0E088E001900D925D
:100960008150E1F708958091790090917A00892B68
:1009700031F010927A001092790081E0089586EBB0
:1009800090E06EEB70E048E050E0ADD308950F9337
:100990001F93DF93CF93CDB7DEB7C954D0400FB6C6
:1009A000F894DEBF0FBECDBF80E005D2BE01675F09
:1009B0007F4F80E0FB01EF93FF9300E810E41023EA
:1009C000A9F00000A59A000000000000000000004F
:1009D00000000000000000000000A59838E03A95F3
:1009E000F1F700000000069561F0E8CFA59A3BE022
:1009F0003A95F1F70000A59800000000069509F06F
:100A0000DDCFA59800E813E01023A9F00000A59A17
:100A100000000000000000000000000000000000D6
:100A200000000000A59838E03A95F1F700000000BA
:100A3000069561F0E8CFA59A3BE03A95F1F7000002
:100A4000A59800000000069509F0DDCFA59800E804
:100A5000182F1023A9F00000A59A00000000000044
:100A60000000000000000000000000000000A59849
:100A700038E03A95F1F700000000069561F0E8CF04
:100A8000A59A3BE03A95F1F70000A5980000000018
:100A9000069509F0DDCFA5980000000000000000D9
:100AA000A59A0000000000000000A59813B3107282
:100AB000E9F330E40FE30A9529F113B31072D9F783
:100AC000C1980000000000000000000000000000CD
:100AD0000000000000000000000000000000000016
:100AE00023B3C19A207221933A9539F00FE30A9506
:100AF00049F023B32072F1F6FACF882705C0C19AD6
:100B0000832F02C088278095FF91EF91C1988F3F76
:100B100021F481E08093C6001BC1FE01319688E07C
:100B2000DF011D928A95E9F7498120E030E0DB0181
:100B300060E870E0F9017096EA0FFB1F808188235E
:100B400039F0CB01022E02C0959587950A94E2F701
:100B5000482B2F5F3F4F2830310561F749834A8189
:100B600020E030E0DE01199660E870E0F901789647
:100B7000EA0FFB1F8081882339F0CB01022E02C0CF
:100B8000959587950A94E2F7482B2F5F3F4F2830C1
:100B9000310561F740954A834B8120E030E0DE016A
:100BA000199660E870E0F901B096EA0FFB1F8081AA
:100BB000882339F0CB01022E02C0959587950A94BF
:100BC000E2F7482B2F5F3F4F2830310561F74B8309
:100BD0004C8120E030E0DE01199660E870E0F90118
:100BE000B896EA0FFB1F8081882311F080E007C0D0
:100BF000CB01022E02C0959587950A94E2F7482B07
:100C00002F5F3F4F2830310551F74C834D8120E055
:100C100030E0DE01199660E870E0F901F096EA0F25
:100C2000FB1F8081882339F0CB01022E02C09595ED
:100C300087950A94E2F7482B2F5F3F4F2830310504
:100C400061F740954D834E8120E030E0DE0119963A
:100C500060E870E0F901F896EA0FFB1F80818823B5
:100C600039F0CB01022E02C0959587950A94E2F7E0
:100C7000482B2F5F3F4F2830310561F740954E8359
:100C80004F8120E030E0DE01199661E070E0F9016B
:100C90003396EA0FFB1F8081882339F0CB01022EA7
:100CA00002C0880F991F0A94E2F7482B2F5F3F4F2D
:100CB0002530310561F720E030E0DE01199660E271
:100CC00070E0F9013996EA0FFB1F8081882339F023
:100CD000CB01022E02C0880F991F0A94E2F7482B1D
:100CE0002F5F3F4F2330310561F74F83488520E068
:100CF00030E0DE01199661E070E0F9013C96EA0F00
:100D0000FB1F8081882339F0CB01022E02C0880F9F
:100D1000991F0A94E2F7482B2F5F3F4F243031058B
:100D200061F789818093B6008A818093B7008B81B7
:100D30008093B8008C818093B9008D818093BA0034
:100D40008E818093BB008F818093BC004093BD0057
:100D5000C75BDF4F0FB6F894DEBF0FBECDBFCF919C
:100D6000DF911F910F9108951092C60010DE90E060
:100D70008091C600882309F491E0892F08951F937C
:100D80001FB7F894B99AC198A598AD9800DE1FBF17
:100D90001F91089586E990E090936A00809369001E
:100DA0009FD1909368008093670085E690E0089556
:100DB00082E190E00895EF92FF920F931F93DF93EB
:100DC000CF93CDB7DEB7C154D0400FB6F894DEBF95
:100DD0000FBECDBFFE013196EF93FF9300E8182FB1
:100DE0001023A9F00000A59A0000000000000000F8
:100DF000000000000000000000000000A59838E09E
:100E00003A95F1F700000000069561F0E8CFA59A49
:100E10003BE03A95F1F70000A59800000000069528
:100E200009F0DDCFA59800000000000000000000E0
:100E30000000000000000000A59A00000000000073
:100E40000000A59830E20FEF0A9529F113B3107254
:100E5000D9F7C19800000000000000000000000069
:100E60000000000000000000000000000000000082
:100E7000000023B3C19A207221933A9539F00FEF05
:100E80000A9549F023B32072F1F6FACF882705C0FE
:100E9000C19A832F02C088278095FF91EF91C19856
:100EA0008F3F21F481E08093D700A8C020E030E09C
:100EB00010E0BF0141E050E0FB01E20FF31F808131
:100EC000882339F0CA01022E02C0880F991F0A94A4
:100ED000E2F7182B2F5F3F4F2430310569F720E0F0
:100EE00030E0BE016F5F7F4F40E150E0F9013C967A
:100EF000E60FF71F8081882339F0CA01022E02C055
:100F0000880F991F0A94E2F7182B2F5F3F4F243068
:100F1000310561F79B85911191E08C85811182E00B
:100F2000682F692B20E030E050E07E010894E11C3E
:100F3000F11CA0E8B0E0F9017096EE0DFF1D808174
:100F4000882339F0CD01022E02C0959587950A9429
:100F5000E2F7582B2F5F3F4F2830310561F720E033
:100F600030E040E07E010894E11CF11CA0E8B0E014
:100F7000F9017896EE0DFF1D8081882339F0CD01AF
:100F8000022E02C0959587950A94E2F7482B2F5FB1
:100F90003F4F2830310561F751585093C7008FE714
:100FA000982F941B9093C8008093C9008093CA0027
:100FB0008093CB008093CC001093CD006093CE0043
:100FC0008D81882319F064606093CE008E81882320
:100FD00029F08091CE0088608093CE008F81882395
:100FE00029F08091CE0080618093CE00888588238F
:100FF00029F08091CE0080628093CE00CF5BDF4FDE
:101000000FB6F894DEBF0FBECDBFCF91DF911F9119
:101010000F91FF90EF90089581E0CDDE08951F932A
:101020001FB7F894B99AC198A598AD98F5DF1FBF7E
:101030001F9108951F93CF93DF9310E0CCE2D1E08E
:1010400011C0FE013197F1F70197D9F71092D7003F
:10105000E3DF8091D700882341F01F5F1F3011F438
:1010600080E004C08CE291E0ECCF81E0DF91CF9191
:101070001F910895009741F0DC01E7ECF0E088E073
:1010800001900D928150E1F7AFECB0E0E7ECF0E0B9
:1010900088E001900D928150E1F7089580918F00D2
:1010A00090919000892B31F01092900010928F0057
:1010B00081E0089587EC90E06FEC70E048E050E04C
:1010C00012D0089586E990E09093800080937F008D
:1010D00007D090937E0080937D008BE790E0089589
:1010E00085E390E00895FB01DC0104C08D9101903F
:1010F000801921F441505040C8F7881B990B08957E
:04110000F894FFCF91
:10110400FFFFFFD25A08000000000000000000BFEB
:1011140006C704B3049F04B40601000800000000DD
:1011240000000000000F080C084E083A081A0801D5
:021134000000B9
:00000001FF
